:020000040800F2
:100000000050002079170008BF170008C11700082A
:10001000C3170008C5170008C71700080000000034
:10002000000000000000000000000000C9170008E8
:10003000CB17000800000000CD170008B50100082C
:10004000D3170008D5170008D7170008D9170008DC
:10005000DB170008DD170008DF170008E1170008AC
:10006000E3170008E5170008E7170008E91700087C
:10007000C10C0008ED170008EF170008F117000881
:10008000F3170008F5170008F7170008F91700081C
:10009000FB170008FD170008FF17000801180008EB
:1000A00003180008051800080718000809180008B8
:1000B0000B1800080D1800080F1800081118000888
:1000C0001318000815180008171800081918000858
:1000D0001B180008AD05000885030008211800085A
:1000E00023180008251800082718000810B5054C2B
:1000F000237833B9044B13B10448AFF300800123D4
:10010000237010BDE002002000000000781F0008EE
:1001100008B5064B1BB106480649AFF300800648F8
:10012000036813B1054B03B1984708BD00000000F8
:10013000781F0008E4020020E00200200000000018
:10014000154B002B08BF134B9D46A3F5803A0021A9
:100150008B460F461348144A121A01F0D3FE0F4B78
:10016000002B00D098470E4B002B00D09847002062
:10017000002104000D000D48002802D00C48AFF308
:10018000008001F099FE2000290000F0FFFB01F043
:100190007FFE00BF000008000050002000000000AB
:1001A00000000000E0020020DC1D00200000000034
:1001B00000000000034B1A6812B11A68013A1A6075
:1001C000704700BFD81D0020084B1B68012B09D0C9
:1001D000074B084A1B68B0FBF3F010601368002B54
:1001E000FCD17047034A1060F8E700BFFC02002012
:1001F00004000020D81D0020044B054A1B6803FBA7
:1002000000F010601368002BFCD170470000002044
:10021000D81D00200128F0B41DD0022823D0164993
:10022000164B64200A2208601A60032042F2107202
:100230001349144B0F68144DB7FBF2F7134A013FF3
:10024000F026002407215F6085F823609C60196018
:100250001060F0BC70470849084B4FF47A721A607E
:1002600008600B4AE4E70449044B64220A241A603C
:100270000C60084ADCE700BF0400002000000020FA
:100280007402002010E000E000ED00E0FC0200201D
:1002900040420F00A086010000F0D2BDF8B5A0F1E9
:1002A0000906032E054602D900242046F8BD00F0B9
:1002B0009BFC00F0A3FB0028F6D02E4F384600F040
:1002C0006DFC3B7804462C4A2C480121222B03600C
:1002D000116001D0282BE8D100F090FB0028E4D079
:1002E000552000F01BFC264F0821224800F048FC56
:1002F000BE2000F013FC3846092100F001FC3B79D8
:10030000C3F341130933AB42CFD000F077FB002891
:10031000CBD0552000F002FC0821164800F030FC3C
:100320004E2000F0FBFB7F2000F0F8FB802000F067
:10033000F5FB700100F0E00000F0F0FB00F05EFB68
:1003400000F05CFB0028B0D0552000F0E7FB094826
:10035000082100F015FC482000F0E0FBFA2501E040
:10036000013D03D000F09EFB0028F9D000F046FBD1
:100370009BE700BF140300200C03002010030020A3
:100380000003002038B5274840F2255101F0C6F996
:1003900020BB244840F2277101F0C0F900B938BDF4
:1003A000204840F2277101F0DFF91F4B1A68002A3C
:1003B00030D01E4A1E4C1168481C8028106008BFAF
:1003C000002054F8211008BF10601A6889B2013A61
:1003D0001A601448BDE8384001F08AB9114840F26B
:1003E000255101F0C1F90F4801F086F9114B1A6847
:1003F0007F2ACED8104A114D1468C0B2611C7F29E3
:10040000116045F8240084BF002111601A68013290
:100410001A60BEE7034840F22771BDE8384001F09A
:1004200049B900BF00440040240500201C050020FD
:100430001C03002020050020280500202C0500209A
:1004400010B582B001A800F021FF0820012100F0C2
:10045000BDFF08240222042301A90548ADF8044089
:100460008DF806208DF8073000F0AEFE02B010BD0A
:10047000000C014030B5314B87B01A680546824206
:100480005AD068461D6000F001FF02A801F0F8F89C
:100490000420012100F09AFF0420012100F096FFC2
:1004A0004FF48040012100F091FF03244FF40072CB
:1004B000182369462248ADF800208DF803308DF8E6
:1004C000024000F081FE4FF48062482369461C48D8
:1004D000ADF800208DF803308DF8024000F074FE76
:1004E0001848012101F00CF900240C2302A9154839
:1004F000ADF812300295ADF80C40ADF80E40ADF8F5
:100500001040ADF8144001F05DF80E48012101F0F3
:10051000C3F80C48012240F2255101F0CBF8252206
:10052000012301A88DF805408DF806408DF80420C0
:100530008DF8073000F030FD07B030BD2C070020EB
:10054000000801400038014030B40E4A13687F2B88
:10055000FCD80D4B0D4D1C68611C7F29196088BFAC
:10056000002145F8240088BF196072B61368013372
:10057000136062B6064840F22771012230BC01F0D8
:1005800099B800BF38090020400B00203007002038
:100590000038014010B50446007828B1FFF7D4FFB9
:1005A00014F8010F0028F9D110BD00BF38B5274855
:1005B00040F2255101F0B2F820BB244840F22771E7
:1005C00001F0ACF800B938BD204840F2277101F0C5
:1005D000CBF81F4B1A68002A30D01E4A1E4C1168F7
:1005E000481C8028106008BF002054F8211008BF64
:1005F00010601A6889B2013A1A601448BDE83840A0
:1006000001F076B8114840F2255101F0ADF80F48DD
:1006100001F072F8114B1A687F2ACED8104A114D9A
:100620001468C0B2611C7F29116045F8240084BFA2
:10063000002111601A6801321A60BEE7034840F2D7
:100640002771BDE8384001F035B800BF00380140DF
:10065000380900203009002030070020340900202C
:100660003C090020400900204FF4E130FFF702BFB1
:100670007F4B2DE9F04F83FB0243D217C2EB631986
:10068000B9F1000F83B006460F4640F3EC804846B0
:1006900001F03AFA82464FF00108404601F034FA80
:1006A000514601F039FB0024054646E0C0F08D803C
:1006B000022A1CD129464FF07E5001F06FF96D4996
:1006C000834601F075FA01F0C3FB6B498DF8040015
:1006D000584601F06DFA01F0BBFB68498DF8050042
:1006E000584601F065FA01F0B3FB8DF806003B5D5A
:1006F000012B7ED040D3022B17D15E49284601F052
:1007000057FA01F0A5FB5C498DF80400284601F07A
:100710004FFA01F09DFB59498DF80500284601F07C
:1007200047FA01F095FB8DF80600204601A9013437
:1007300000F05CFB902C00F08880325D0023012AE1
:100740008DF804308DF805308DF80630AED129468D
:100750004FF07E5001F022F94949834601F028FA12
:1007600001F076FB47498DF80400584601F020FA65
:1007700001F06EFB4449B1E70021284601F018FA68
:1007800083469DF8040001F0BFF9594601F008F9CD
:1007900001F05EFB8DF804009DF8050001F0B4F94E
:1007A0000146584601F0FCF801F052FB8DF80500B7
:1007B0009DF8060001F0A8F90146584601F0F0F84E
:1007C00001F046FB8DF80600AFE729464FF07E505A
:1007D00001F0E4F8002101F0EBF901F039FB3B5D99
:1007E000C0B2012B8DF804008DF805008DF80600CD
:1007F00080D19DF8040001F087F9214983462846FD
:1008000001F0D6F90146584601F0CAF801F020FB84
:100810008DF804009DF8050001F076F9194983462A
:10082000284601F0C5F90146584601F0B9F801F033
:100830000FFB8DF805009DF8060001F065F91249DF
:100840008346284601F0B4F9B6E7204600F046FAA0
:1008500008F101086420FFF7CFFCC145BFF61DAFCA
:1008600003B0BDE8F08F4FF07E5A4FF0010912E758
:100870001F85EB510000A040000010410000234301
:100880000000714300004D430000704270B50E4CF3
:100890000E4E0F4D304621464FF4FA72FFF7E8FE38
:1008A000204629464FF4FA72FFF7E2FE2846214619
:1008B0004FF4FA72FFF7DCFE204631464FF4FA722D
:1008C000BDE87040FFF7D4BE08000020640100209E
:1008D000D801002038B5124C124D21460022204686
:1008E000FFF7C6FE4FF4FA60FFF786FC2046294664
:1008F0006422FFF7BDFE284621466422FFF7B8FEBA
:10090000204629466422FFF7B3FE2846214664228A
:10091000FFF7AEFEBDE838404FF47A70FFF76CBCCD
:100920007C000020F000002010B403460022C17BB0
:100930005C7E0132C473597690F8251093F82F40ED
:10094000052A80F8254083F82F1090F83B1093F883
:10095000454000F1010080F83A4083F8451090F8D6
:10096000501093F85B4003F1FF3380F8504083F858
:100970005C1090F8661093F8724080F8664083F837
:100980007210D4D15DF8044B704700BF10B500F071
:100990004FFF00F0D1FF0120014600F017FD0121BB
:1009A000134800F087FCFFF75FFEFFF749FD00F0FA
:1009B00043F900F065F90120FFF72CFCFFF76CFC10
:1009C00000F07AF900F03CFA0A48FFF7ADFF002486
:1009D0000948FFF7A9FF012C04DDFFF77BFF002486
:1009E000FFF778FF0134FFF751FF012CF5DCF9E741
:1009F000000230007C000020F0000020F8B56420E8
:100A0000FFF7E2FB20210022244800F04DFC4FF4C8
:100A10000C70FFF7D9FB21482021012200F044FC93
:100A20001F4D1420FFF7D0FB00274FF496732B6067
:100A30003E4603E006B92E682C686CB117482021A9
:100A400000F02CFC0028F5D0002EF5D0002FF3D1BB
:100A50002F682C68002CF1D132208EB187B1FFF7BE
:100A6000B3FB20210D4800F019FCF61B0546782049
:100A7000FFF7AAFB1E2E0ED96B1E58425841F8BD37
:100A8000FFF7A2FB2021054800F008FC7820FFF7C3
:100A90009BFB0020F8BD2046F8BD00BF000C0140C4
:100AA000D81D002010B50E4C20212046002200F059
:100AB000FBFB0520FFF788FB01222046202100F0E8
:100AC000F3FB0A20FFF780FB2021204600F0E6FB25
:100AD00004463220FFF778FB631E5842584110BD90
:100AE000000C014070B5082401250026FFF7DAFF4D
:100AF0006B0000B12E43013CDDB2F7D1304670BD32
:100B000038B54D1E0446EDB239B101350544FFF745
:100B1000E9FF04F8010BAC42F9D138BD70B50646C7
:100B20000825012411E0002200F0BEFB0520FFF79C
:100B30004BFB12482021012200F0B6FB5020FFF7AA
:100B400043FB6400013DE4B216D014EA06024FF004
:100B500020010A48E7D100F0A7FB5020FFF734FB43
:100B600006482021012200F09FFB0520FFF72CFB07
:100B70006400013DE4B2E8D170BD00BF000C01404B
:100B800038B54D1E0446EDB239B10135054414F8AF
:100B9000010BFFF7C3FFAC42F9D138BD38B50446AD
:100BA000FFF72CFF70B13320FFF7B8FF04F1080501
:100BB000FFF798FF04F8010BAC42F9D1FFF71EFFD5
:100BC000012038BD234603F8010B0133607003F8A0
:100BD000010B03F8010B03F8010B03F8010B03F8F9
:100BE000010B187038BD00BF30B5114B83B01A68C7
:100BF0000AB103B030BD012401A81C6000F046FB1F
:100C00002146202000F0E2FB2025032301A9142225
:100C100008488DF807208DF80630ADF8045000F034
:100C2000D3FA29462246034800F03EFB03B030BD0C
:100C3000440B0020000C014010B582B001A800F068
:100C400025FB0820012100F0C1FB01240222102312
:100C500001A908488DF806208DF80730ADF804404A
:100C600000F0B2FA0448FFF795FC0448FFF792FC45
:100C700002B010BD000C0140301F0008441F0008E6
:100C800010B5094C2368012B0CD001210A460748F6
:100C900000F00AFB0648FFF77DFC0648FFF77AFCE8
:100CA0000123236010BD00BF4C020020000C014056
:100CB000481F0008441F00080920FFF7EFBA00BFD3
:100CC00008B5202000F068FA28B1202000F072FA60
:100CD000014B00221A6008BD480B00202DE9F047A7
:100CE000DFF804E10746DEF80030002BFBD1002FCF
:100CF0006ED04FEA4708384808EB070C3749844460
:100D0000182610F802ACA6F11803A6F110098022EB
:100D100012EA0A0F03F101030CBF22253A25CC1871
:100D20004B454FEA520204F8015CF1D110F803ACD4
:100D3000A6F10809802212EA0A0F03F101030CBF91
:100D400022253A25CC184B454FEA520204F8015CA3
:100D5000F1D110F8019C802212EA090F03F101037E
:100D60000CBF22253A25CC189E424FEA520204F8C5
:100D7000015CF1D10330604506F11806C1D10022B3
:100D80000B44104698540132302AFBD101241448F8
:100D90000021CEF8004000F0D7FB1248002100F0FF
:100DA000E3F907EB0801C900303189B20D4800F0C2
:100DB000F1F922460B48022100F0E2F921460948E8
:100DC00000F0D2F921460648BDE8F04700F0BCBB70
:100DD00002493B46B846D2E74F0B0020580D002091
:100DE000002C01401C000240480B0020AD2809D80F
:100DF0000A78054B00EB40001A544A7818444270B8
:100E00008B788370704700BF4C0B0020F0B469B141
:100E10000A4D01EB410700230678EC18EE544678A2
:100E2000033366708678BB42A670F5D10AB9F0BC70
:100E300070470846F0BCFFF751BF00BF4C0B0020C5
:100E40002DE9F0414E4D94B0002468462C6000F02E
:100E50001DFA0420012100F0B9FA4FF48077032332
:100E60001822694647488DF802308DF80320ADF806
:100E7000007000F0A9F922463946424800F014FA01
:100E800002A800F04DFB05A800F054FB4FF40060F1
:100E9000012100F09BFA0120014600F08BFA5B2350
:100EA00002A939480126ADF80C30ADF80840ADF87C
:100EB0000E40ADF80A4000F095FA602305A93248CB
:100EC000ADF81430ADF81660ADF81A40ADF81C401E
:100ED00000F0DEFA2C48082100F06CFB31462A486D
:100EE00000F05AFB3146284800F03CFB32464FF4F4
:100EF0000071254800F046FB0C2301A88DF8043052
:100F00008DF807608DF805408DF8064000F044F834
:100F100009A800F01BF921461C4800F025F91B48E0
:100F200000F072F8DFF86880DFF868C04FF4845E84
:100F30004FF44052102309A9802614480F971194AA
:100F400010940D941394CDF82480CDF828C0CDF8DA
:100F500030E00E9612920B9300F0D8F88DF82440F2
:100F60008DF825408DF826402B68002BFCD109A870
:100F7000AE210122FFF74AFF14B0BDE8F08100BFA7
:100F8000480B002000080140002C01401C000240DA
:100F9000342C0140580D0020C37830B45BB903787D
:100FA000012103F01F0291405B09154A203342F8EA
:100FB000231030BC7047134B4478DB680F22DB43AF
:100FC000C3F30223C3F1040122FA03F38C408578B2
:100FD000017803EA0502224301F160431201D2B213
:100FE00003F5614383F800230378012103F01F0216
:100FF0009140034A5B0942F8231030BC704700BFA0
:1010000000E100E000ED00E0036833494FF6FE72B6
:101010001A4088424FF0000302600360436083601F
:10102000C36044D02D4B984225D02D4B984230D0F0
:101030002C4B984234D02C4B984223D02B4B9842C7
:101040003BD02B4B98420FD02A4B98423CD02A4B96
:10105000984210D0294B98421BD0294B98421FD060
:10106000284B98420ED0704753F87C2C42F07062A7
:1010700043F87C2C704753F8182C42F0F00243F8E8
:10108000182C704753F8542C42F4702243F8542C17
:10109000704753F82C2C42F4706243F82C2C7047A4
:1010A00053F8402C42F4704243F8402C7047164BE2
:1010B0005A6842F00F025A60704753F8682C42F4A5
:1010C000700243F8682C704753F8042C42F00F026A
:1010D00043F8042C704700BF080002401C00024087
:1010E0003000024044000240580002406C000240C0
:1010F00080000240080402401C0402403004024008
:101100004404024058040240000002408A68F0B4DF
:101110000C6A0B6914434A691C438B69CE692243EC
:1011200007684D6A13438C6A1E43354327F4FF4317
:101130002C4323F0700323430360CB68F0BC43606F
:101140000B6883604B68C360704700BF0023036077
:1011500043608360C360036143618361C361036271
:1011600043628362704700BF29B902684FF6FE737D
:10117000134003607047036843F001030360704746
:1011800003681AB923EA010101607047194301603D
:10119000704700BF41607047C3004CBF034B044B16
:1011A0001B6803420CBF002001207047000402406E
:1011B00000000240C3004CBF014B024B5860704717
:1011C0000004024000000240CB782DE9F00303F058
:1011D0000F06DB0648BF8B780A8848BF1E4312F013
:1011E000FF0F26D00768002301254FF00F0803E00A
:1011F0000133082B1BD00A8805FA03F42240A242CF
:10120000F6D19C0008FA04F906FA04F491F803C038
:1012100027EA0907BCF1280F47EA040734D0BCF1DC
:10122000480F03F1010308BF0261082BE3D10760F7
:101230000A88FF2A25D94768002301254FF00F0CA3
:1012400003E00133082B1BD00A8803F1080405FAD8
:1012500004F42240A242F4D19C000CFA04F906FAEC
:1012600004F8CC780133282C04BF4261CC7827EAFB
:101270000907482C08BF0261082B47EA0807E3D199
:101280004760BDE8F00370474261B1E74FF6FF7178
:101290000222042301808270C37070478368194260
:1012A0000CBF0020012070470AB9416170470161FD
:1012B000704700BF30B40028184B00F44012B4BF90
:1012C000DB695B68B2F5401F84B21FD0C20214D53F
:1012D000C0F30342032505FA02F223EA020343F0B6
:1012E000706319B1420D1201944023430B4A002848
:1012F000B4BFD361536030BC7047420D120104FA91
:1013000002F223EA020343F07063EAE7034A23F0A0
:101310007063556825F070655560E2E70000014094
:1013200030B41F494B6803F00C03042B01D0082B89
:1013300020D01C4A02601A4B1B495D681B4CC5F348
:1013400003154D5DEA4042605D68C5F302254D5DC1
:1013500022FA05F585605D68C5F3C225495DCA407E
:10136000C2605B68C3F38133E35C30BCB2FBF3F271
:10137000026170474A684B68C2F38342DC0302F1A2
:10138000020207D54B689B0304D4064B03FB02F211
:101390000260D0E7064B03FB02F20260CBE700BF1E
:1013A0000010024000127A00540200205002002077
:1013B00000093D00044B5A6919B922EA000058613E
:1013C000704710435861704700100240044B9A69FF
:1013D00019B922EA0000986170471043986170477C
:1013E00000100240274A038890429BB212D002F5B7
:1013F000006290420ED0B0F1804F0BD0A2F598322F
:10140000904207D002F58062904203D002F58062DC
:10141000904203D14A8823F0700313431A4A904242
:1014200027D002F58062904223D0CA8823F440730B
:101430009BB2134303808A88124B82850A889842A4
:10144000028511D0114B98420ED003F540639842AB
:101450000AD003F58063984206D003F58063984272
:1014600002D00123838270470B7A03860123838293
:10147000704703808B8883850B88038501238382D3
:10148000704700BF002C01400010004000340140B4
:10149000038CF0B423F001031B041B0C0384028CA7
:1014A0000D8984884F88038B2F4322F0020223F09A
:1014B00073031A4D12041B040E88120CBFB21B0CCE
:1014C000A84247EA0202A4B243EA060316D005F591
:1014D0000065A84212D005F54065A8420ED005F57A
:1014E0008065A8420AD005F58065A84206D08480B0
:1014F0000383CB88F0BC8386028470474E89CF89F2
:101500008D8922F0080232433D438E8824F44074D2
:1015100022F00402ADB232432C43E8E7002C014034
:1015200000234FF6FF7282800380C38043800372E2
:10153000704700BF0023038043808380C380038102
:1015400043818381C3817047038829B923F0010354
:101550001B041B0C038070479BB243F00103038004
:10156000704700BFB0F8443021B9C3F30E03A0F8B0
:10157000443070476FEA43436FEA53439BB2A0F88D
:101580004430704783899BB21AB923EA01018181F3
:101590007047194381817047038829B923F080037C
:1015A0001B041B0C038070479BB243F08003038035
:1015B000704700BF038B23F008031B041B0C194367
:1015C0000183704730B5038ACA889BB223F4405325
:1015D00013430382828904460B8988880D4692B2A0
:1015E0004989034322F4B0520B4322F00C02134307
:1015F0009BB2A381A38AAA899BB223F4407387B0CC
:101600001343A38201A8FFF78BFEA189049A1A480D
:10161000039B09B2844208BF13462A68002903EBE2
:101620008303B4BF5200920003EB83031349B3FB5F
:10163000F2F3A1FB0352A089520900B264250028ED
:1016400002FB15334FEA02120ADB1B013233A1FB06
:101650000351C1F343110A4392B2228107B030BD56
:10166000DB003233A1FB0301C1F342110A4392B202
:10167000228107B030BD00BF003801401F85EB510B
:1016800000234FF416510C22016042818380C380F5
:1016900003818381704700BF838929B923F40053F4
:1016A0001B041B0C838170479BB243F4005383815E
:1016B000704700BF01F01F0310B4C1F342110124B1
:1016C000A14204FA03F310D002290CBF10301430E9
:1016D00004682AB924EA030303605DF8044B7047E9
:1016E000234303605DF8044B70470C30F0E700BF04
:1016F000C1F30801818070478088C0F308007047FB
:10170000838919B9C3F30E03838170476FEA43439A
:101710006FEA53439BB28381704700BF10B4C1F39B
:101720004213012401F01F02A34204FA02F217D06F
:10173000022B0CBF038A838A9BB21340028892B2A9
:1017400053B1090A012303FA01F111420CBF002031
:1017500001205DF8044B704718465DF8044B704754
:1017600083899BB21340E9E7090A01238B40DB43DD
:101770009BB20380704700BF0649074A074B9A4255
:10178000BEBF51F8040B42F8040BF8E70448804749
:1017900004480047841F000800000020E0020020E9
:1017A00031180008410100081F49204A002301E0C8
:1017B00041F8043B9142FBD3FFF7E8F8FEE7FEE770
:1017C000FEE7FEE7FEE7FEE7FEE7FEE7FEE7FEE7F1
:1017D000FEE7FEE7FEE7FEE7FEE7FEE7FEE7FEE7E1
:1017E000FEE7FEE7FEE7FEE7FEE7FEE7FEE7FEE7D1
:1017F000FEE7FEE7FEE7FEE7FEE7FEE7FEE7FEE7C1
:10180000FEE7FEE7FEE7FEE7FEE7FEE7FEE7FEE7B0
:10181000FEE7FEE7FEE7FEE7FEE7FEE7FEE7FEE7A0
:10182000FEE7FEE7FEE7FEE7E0020020DC1D002009
:1018300010B43D4B3D4A196883B041F00101196075
:10184000596800200A405A6019684FF41F0421F0BB
:10185000847121F48031196019681A4621F48021BD
:101860001960596821F4FE0159609C600090019054
:10187000196841F48031196003E0009BB3F5A06F53
:1018800009D0136803F400330193009B01330093E4
:10189000019B002BF1D0244B1B6813F4003318BFBD
:1018A00001230193019B012B07D0214B4FF00062D4
:1018B0009A6003B05DF8044B70471E4A1A4B1068DB
:1018C000194640F010001060106820F0030010600E
:1018D000106840F0020010605A685A605A685A60F6
:1018E0005A6842F480625A605A6822F47C125A6044
:1018F0005A6842F4E8125A601A6842F080721A601C
:101900000B68094A9B01FBD55368114623F003037A
:101910005360536843F0020353604B6803F00C03B9
:10192000082BFAD1C1E700BF001002400000FFF809
:1019300000ED00E000200240114B5A6802F00C025A
:10194000082A0ED15A685968C2F38342C90302F1CA
:10195000020211D55B689B030ED40A4B03FB02F213
:1019600000E0084A064B08485968084BC1F30311C8
:10197000415CCA401A607047054B03FB02F2F1E775
:101980000010024000127A0064020020740200205D
:1019900000093D0080F0004002E000BF81F00041FE
:1019A00042001FBF5FEA410392EA030F7FEA226C05
:1019B0007FEA236C6AD04FEA1262D2EB1363C1BF95
:1019C000D218414048404140B8BF5B42192B88BF04
:1019D000704710F0004F40F4000020F07F4018BF27
:1019E000404211F0004F41F4000121F07F4118BF47
:1019F000494292EA030F3FD0A2F1010241FA03FCEF
:101A000010EB0C00C3F1200301FA03F100F00043D6
:101A100002D5494260EB4000B0F5000F13D3B0F19E
:101A2000807F06D340084FEA310102F10102FE2A0D
:101A300051D2B1F1004F40EBC25008BF20F001007D
:101A400040EA03007047490040EB000010F4000F2B
:101A5000A2F10102EDD1B0FA80FCACF1080CB2EBBE
:101A60000C0200FA0CF0AABF00EBC250524218431D
:101A7000BCBFD0401843704792F0000F81F40001C2
:101A800006BF80F400000132013BB5E74FEA410395
:101A90007FEA226C18BF7FEA236C21D092EA030F01
:101AA00004D092F0000F08BF0846704790EA010F7B
:101AB0001CBF0020704712F07F4F04D1400028BFA8
:101AC00040F00040704712F100723CBF00F500008A
:101AD000704700F0004343F0FE4040F400007047C0
:101AE0007FEA226216BF08467FEA2363014642026C
:101AF00006BF5FEA412390EA010F40F4800070477F
:101B00004FF0000304E000BF10F0004348BF404224
:101B10005FEA000C08BF704743F0964301464FF060
:101B200000001CE050EA010208BF70474FF00003BC
:101B30000AE000BF50EA010208BF704711F00043FD
:101B400002D5404261EB41015FEA010C02BF8446CD
:101B50000146002043F0B64308BFA3F18053A3F52C
:101B60000003BCFA8CF2083AA3EBC25310DB01FA73
:101B700002FC634400FA02FCC2F12002BCF1004FF7
:101B800020FA02F243EB020008BF20F00100704788
:101B900002F1200201FA02FCC2F1200250EA4C00DC
:101BA00021FA02F243EB020008BF20EADC70704722
:101BB0004FF0FF0C1CEAD0521EBF1CEAD15392EA30
:101BC0000C0F93EA0C0F6FD01A4480EA010C40020C
:101BD00018BF5FEA41211ED04FF0006343EA501066
:101BE00043EA5111A0FB01310CF00040B1F5000FA8
:101BF0003EBF490041EAD3715B0040EA010062F157
:101C00007F02FD2A1DD8B3F1004F40EBC25008BF40
:101C100020F00100704790F0000F0CF0004C08BF5E
:101C200049024CEA502040EA51207F3AC2BFD2F12B
:101C3000FF0340EAC250704740F400004FF0000339
:101C4000013A5DDC12F1190FDCBF00F00040704773
:101C5000C2F10002410021FA02F1C2F1200200FAB1
:101C600002FC5FEA310040F1000053EA4C0308BF78
:101C700020EADC70704792F0000F00F0004C02BFC9
:101C8000400010F4000F013AF9D040EA0C0093F044
:101C9000000F01F0004C02BF490011F4000F013B9E
:101CA000F9D041EA0C018FE70CEAD15392EA0C0F0C
:101CB00018BF93EA0C0F0AD030F0004C18BF31F077
:101CC000004CD8D180EA010000F00040704790F04D
:101CD000000F17BF90F0004F084691F0000F91F0F1
:101CE000004F14D092EA0C0F01D142020FD193EAB7
:101CF0000C0F03D14B0218BF084608D180EA01003F
:101D000000F0004040F0FE4040F40000704740F01A
:101D1000FE4040F4400070474FF0FF0C1CEAD052E8
:101D20001EBF1CEAD15392EA0C0F93EA0C0F69D044
:101D3000A2EB030280EA010C49024FEA402037D0AF
:101D40004FF0805343EA111143EA10130CF00040A6
:101D50008B4238BF5B0042F17D024FF4000C8B4296
:101D600024BF5B1A40EA0C00B3EB510F24BFA3EB76
:101D7000510340EA5C00B3EB910F24BFA3EB910346
:101D800040EA9C00B3EBD10F24BFA3EBD10340EAA0
:101D9000DC001B0118BF5FEA1C1CE0D1FD2A3FF6E6
:101DA00050AF8B4240EBC25008BF20F0010070479B
:101DB0000CF0004C4CEA50207F32C2BFD2F1FF033E
:101DC00040EAC250704740F400004FF00003013A6F
:101DD00037E792F0000F00F0004C02BF400010F413
:101DE000000F013AF9D040EA0C0093F0000F01F027
:101DF000004C02BF490011F4000F013BF9D041EA49
:101E00000C0195E70CEAD15392EA0C0F08D142027B
:101E10007FF47DAF93EA0C0F7FF470AF084676E74E
:101E200093EA0C0F04D14B023FF44CAF08466EE727
:101E300030F0004C18BF31F0004CCAD130F00042F5
:101E40007FF45CAF31F000437FF43CAF5FE700BF4D
:101E500042000ED2B2F1FE4F0BD34FF09E03B3EB14
:101E6000126209D44FEA002343F0004323FA02F040
:101E700070474FF00000704712F1610F01D142022C
:101E800002D14FF0FF3070474FF00000704700BFA5
:101E900008B5074B044613B10021AFF30080054B92
:101EA0001868836A03B19847204600F033F800BFF2
:101EB00000000000741F000870B50E4B0E4D00248A
:101EC000ED1AAD101E46AC4204D056F824209047BF
:101ED0000134F8E700F020F8084D094B0024ED1A12
:101EE000AD101E46AC4204D056F824209047013471
:101EF000F8E770BDD8020020D8020020DC020020E4
:101F0000D802002002440346934202D003F8011B8A
:101F1000FAE77047FEE70000F8B500BFF8BC08BC60
:101F20009E467047F8B500BFF8BC08BC9E46704797
:101F3000706F7765725F696E697428292063616CC0
:101F40006C6564000D0A0000737769746368696EDC
:101F50006720706F776572206F6E00007377697409
:101F60006368696E6720706F776572206F666600C0
:0C1F700043000000780200200000000088
:081F7C00C4E1FF7F0100000039
:101F8400E803000001000000000000000000000061
:101F9400000100000000000000010000000000013A
:101FA400000000000000010101000000000000002A
:101FB4000101010101000000000100010101010112
:101FC4000001000000000101010101000000000007
:101FD40000000101010000000000000100000000F9
:101FE40000010000000000000001000000000000EB
:101FF40000000000000000000000000000000000DD
:1020040000000000000000000000000002020200C6
:1020140000000000000002020202020002020000AE
:102024000002020202020202020200000202020292
:10203400020202020202000202020202020202027E
:10204400020000020202020202020200000000007A
:10205400000000000000000000000000000000007C
:10206400000000000000000000000000000000006C
:10207400000000000000000000000000000000005C
:10208400020202000000000000000202020202003C
:102094000202000000020202020202020202000026
:1020A4000202020201010102020200020202010113
:1020B4000102020202000002020101020202020005
:1020C4000000000000010100000000000000000109
:1020D40001000000000000000001010000000000F9
:1020E40000000000000000000000000000000000EC
:1020F40000000000000000000000000000000000DC
:1021040000000101010000000000000001010101C4
:1021140001000000000000010101010100000000B5
:1021240000000101010101000000000000000101A4
:10213400010000000000000000000000000000009A
:10214400000000000000000000000000000000008B
:10215400000000000000000000000000000100007A
:102164000001000000010000000100000000000167
:102174000000000000000101010000000000000058
:10218400010101010100000001010001010101013F
:102194000001010000000101010101000000000034
:1021A4000000010101000000000000010000000027
:1021B4000001000000010000000100000001000017
:1021C400000000000100000000000000FF0000000B
:1021D40002040608000000000102030401020304D3
:1021E40006070809000000000000000001020304C3
:1021F4000607080900A24A040000000000000000CD
:1022040000000000000000000000000000000000CA
:102214000000000000000000701F00080000000023
:1022240000000000000000000000000000000000AA
:10223400000000000000000000000000000000009A
:10224400000000000000000000000000000000008A
:10225400000000000000000011010008ED0000086B
:0400000508000000EF
:00000001FF
